:100000000C9435000C945D000C945D000C945D0024
:100010000C945D000C945D000C945D000C945D00EC
:100020000C945D000C945D000C945D000C945D00DC
:100030000C945D000C945D000C945D000C945D00CC
:100040000C9448050C945D000C945D000C945D00CC
:100050000C945D000C945D000C945D000C945D00AC
:100060000C945D000C945D00B80611241FBECFEF08
:10007000D8E0DEBFCDBF11E0A0E0B1E0EEEDFEE0E4
:1000800002C005900D92A232B107D9F721E0A2E299
:10009000B1E001C01D92AD36B207E1F710E0C5E353
:1000A000D0E004C02197FE010E945307C433D1075A
:1000B000C9F70E9492050C946D070C9400003FB79D
:1000C000F89480914C0190914D01A0914E01B09116
:1000D0004F0126B5A89B05C02F3F19F00196A11D21
:1000E000B11D3FBFBA2FA92F982F8827820F911DCE
:1000F000A11DB11DBC01CD0142E0660F771F881F15
:10010000991F4A95D1F708953F924F925F926F924F
:100110007F928F929F92AF92BF92CF92DF92EF9297
:10012000FF920F931F93CF93DF9300D01F92CDB711
:10013000DEB7F82E80915D0190915E01A0915F0184
:10014000B0916001892B8A2B8B2BE9F00E945F0014
:100150000091690110916A0120916B0130916C014D
:10016000DC01CB01801B910BA20BB30B00915D0155
:1001700010915E0120915F0130916001801791071D
:10018000A207B307B8F20E945F0060936901709301
:100190006A0180936B0190936C01E0916501F0918D
:1001A0006601309759F04091610150916201609170
:1001B0006301709164018F2D0995F82E00916701FC
:1001C000109168014F2C512C612C712C01151105D7
:1001D00009F461C0D8011C96EC901C9780915B01DA
:1001E00090915C018436910510F41C961C92D80104
:1001F000ED91FC91A280B38019821A821B82F110CA
:1002000014C0F80145855685628173819E012F5F78
:100210003F4FC801F5010995D8011C96EC921C9737
:1002200014960D911C911597D1CFF8013996CE01F6
:1002300001966C0148019CE0890E911CDF01139727
:100240003C902191332001F12223F1F0822F90E0A4
:10025000A0E0B0E09C01AD012F5F3F4F4F4F5F4FDB
:10026000C301B2010E94C8069B01AC01832D90E03E
:10027000A0E0B0E0BC01CD016F5F7F4F8F4F9F4F7B
:100280000E94C806D6018C93BFEFCB1ADB0AE81593
:10029000F905A1F6B6CF80915801909159019C01C2
:1002A0002F5F3F4F309359012093580149970CF429
:1002B00047C08FB7F89400915001109151012091DF
:1002C0005201309153018FBFE0915801F0915901D3
:1002D00088EE93E0E89FB001E99F700DF89F700DE4
:1002E0001124072E000C880B990BC0905401D0905C
:1002F0005501E0905601F0905701A90198012C1981
:100300003D094E095F090E94EC0630935C01209381
:100310005B0110925901109258012FB7F894809107
:10032000500190915101A0915201B09153012FBF02
:100330008093540190935501A0935601B0935701B7
:100340000F900F900F90DF91CF911F910F91FF9021
:10035000EF90DF90CF90BF90AF909F908F907F9065
:100360006F905F904F903F9008958F929F92AF92C1
:10037000BF92CF92DF92EF92FF926B017C010E94BD
:100380005F004B015C01C114D104E104F104F1F000
:100390000E945F00DC01CB0188199909AA09BB09F9
:1003A000883E9340A105B10570F321E0C21AD1083F
:1003B000E108F10888EE880E83E0981EA11CB11CAC
:1003C000C114D104E104F10419F7DDCFFF90EF90DF
:1003D000DF90CF90BF90AF909F908F900895EF9255
:1003E000FF920F931F93CF93DF93EC019091230122
:1003F0009F5F292F27702093230190FF02C090E870
:1004000001C090E021FD9064247009F0906220E129
:10041000290FFE013C967E018FE0E80EF11C00E002
:1004200011E06191662331F070E0C8010E94D806A6
:100430006F5F01C060E0DF0114976C93322F369F2D
:10044000030E30E0311D1124CF010797311103C095
:10045000EC01188203C03150EC013883662311F09F
:1004600061506C93EE15FF05E1F6DF91CF911F917E
:100470000F91FF90EF9008954F925F926F927F924D
:100480008F92AF92BF92CF92EF92FF920F931F93F2
:10049000CF93DF933C01EB010E945F00F3012785BE
:1004A0003089621B730B6A307105B0F3F894E881F0
:1004B000F9815BB150688BB18F778BB96A859F8169
:1004C000262F291B922F2F83BF844A805B807D8536
:1004D000FC84EE847F5FF394E3943E814885A98495
:1004E000CB841181D20120E0C32F022F322F318122
:1004F000112788943111390F08F43FEF91958894B2
:1005000070FD130F1795889471FD130F179588943C
:1005100072FD130F1795889473FD130F1795889428
:1005200074FD130F1795889475FD130F1795889414
:1005300076FD130F1795889477FD130F1795889400
:10054000232F7111212F960F122F002C5BB900C0A1
:1005500017FF8BB930812227889400C000C0002C7F
:100560008BB931113C0F00C0002C5BB900C016FFE5
:100570008BB908F43FEFC195889400C000C0002CEF
:100580008BB9F0FC230F00C0002C5BB900C015FF35
:100590008BB927958894F1FC230F00C000C0002C74
:1005A0008BB92795889400C0002C5BB900C014FF5C
:1005B0008BB9F2FC230F2795889400C000C0002C53
:1005C0008BB9F3FC230F00C0002C5BB900C013FFF4
:1005D0008BB927958894F4FC230F00C000C0002C31
:1005E0008BB92795889400C0002C5BB900C012FF1E
:1005F0008BB9F5FC230F2795889400C000C0002C10
:100600008BB9F6FC230F00C0002C5BB900C011FFB2
:100610008BB927958894F7FC230F00C000C0002CED
:100620008BB92795889400C0002C5BB900C010FFDF
:100630008BB9132FF110122FCA0D00C000C0002C6F
:100640008BB900C000C0002C5BB900C017FF8BB98C
:1006500032812227889400C000C0002C8BB9311150
:10066000340F00C0002C5BB900C016FF8BB908F432
:100670003FEFEB0DF11D00C000C0002C8BB9E0FC7A
:10068000230F00C0002C5BB900C015FF8BB9279564
:100690008894E1FC230F00C000C0002C8BB9279583
:1006A000889400C0002C5BB900C014FF8BB9E2FC39
:1006B000230F2795889400C000C0002C8BB9E3FC61
:1006C000230F00C0002C5BB900C013FF8BB9279526
:1006D0008894E4FC230F00C000C0002C8BB9279540
:1006E000889400C0002C5BB900C012FF8BB9E5FCF8
:1006F000230F2795889400C000C0002C8BB9E6FC1E
:10070000230F00C0002C5BB900C011FF8BB92795E7
:100710008894E7FC230F00C000C0002C8BB92795FC
:10072000889400C0002C5BB900C010FF8BB9132F58
:10073000E110122F419500C000C0002C8BB94C0D68
:1007400000C000C05BB900C017FF8BB93181222700
:10075000889400C000C0002C8BB93111390F00C043
:10076000002C5BB900C016FF8BB908F43FEF9195E0
:10077000889400C000C0002C8BB970FD230F00C00E
:10078000002C5BB900C015FF8BB92795889471FDCB
:10079000230F00C000C0002C8BB92795889400C09F
:1007A000002C5BB900C014FF8BB972FD230F279595
:1007B000889400C000C0002C8BB973FD230F00C0CB
:1007C000002C5BB900C013FF8BB92795889474FD8A
:1007D000230F00C000C0002C8BB92795889400C05F
:1007E000002C5BB900C012FF8BB975FD230F279554
:1007F000889400C000C0002C8BB976FD230F00C088
:10080000002C5BB900C011FF8BB92795889477FD48
:10081000230F00C000C0002C8BB92795889400C01E
:10082000002C5BB900C010FF8BB9132F7111122F70
:10083000960F00C000C0002C8BB9119709F086CE2E
:1008400020EE31E0D2010E942D07DC01CB01F4E063
:10085000B695A79597958795FA95D1F720E030E062
:10086000A9016AE9469E040C411D569E400D511D8A
:100870001124450D511D840F951FA11DB11D893EE9
:1008800043E09407A105B10508F434C0885E9340A5
:10089000A109B10942E0B695A795979587954A9524
:1008A000D1F747E0849F080E211D949F200D311D34
:1008B0001124290F311D6091220170E0860F971FCE
:1008C000820F931F4091500150915101609152014C
:1008D00070915301292F3327420F531F611D711D42
:1008E0004093500150935101609352017093530112
:1008F0008093220178940E945F00F301708B6787D8
:10090000DF91CF911F910F91FF90EF90CF90BF900B
:10091000AF908F907F906F905F904F90089580E997
:1009200091E00895579A08950F931F93CF93DF9303
:10093000CDB7DEB762970FB6F894DEBF0FBECDBF5E
:100940008C01F901DC011C968C917A8369835C83AC
:100950004B835E834D8390819D8791819E87928199
:100960009F87813029F4CE0101960E94EF0106C0D5
:100970001C861B861A86198618861F8283E0888B40
:100980001A8A198AD801ED91FC910484F585E02D2D
:10099000BE016F5F7F4FC801099562960FB6F8944C
:1009A000DEBF0FBECDBFDF91CF911F910F91089594
:1009B0000F931F93CF93DF93CDB7DEB762970FB638
:1009C000F894DEBF0FBECDBF8C01F901DC011C968F
:1009D0008C917A8369835C834B835E834D839081A2
:1009E0009D8791819E8792819F87813029F4CE01D6
:1009F00001960E94EF0106C01C861B861A86198686
:100A000018861F82188A1A8A198AD801ED91FC91DA
:100A10000484F585E02DBE016F5F7F4FC801099505
:100A200062960FB6F894DEBF0FBECDBFDF91CF91B7
:100A30001F910F91089580E090E00895FC01858555
:100A400096850895CF93DF9300D000D000D0CDB726
:100A5000DEB7AB011C821D821E82DC01ED91FC9190
:100A60000190F081E02D19821A821B829E012F5F76
:100A70003F4FBE016C5F7F4F099526960FB6F894E5
:100A8000DEBF0FBECDBFDF91CF9108950E946807F2
:100A90001F920F920FB60F9211242F933F938F93B3
:100AA0009F93AF93BF938091500190915101A0917A
:100AB0005201B091530130914B0123E0230F2D37A8
:100AC00020F40196A11DB11D05C026E8230F029652
:100AD000A11DB11D20934B018093500190935101B2
:100AE000A0935201B093530180914C0190914D011C
:100AF000A0914E01B0914F010196A11DB11D8093AF
:100B00004C0190934D01A0934E01B0934F01BF91C2
:100B1000AF919F918F913F912F910F900FBE0F90AA
:100B20001F901895789484B5826084BD84B58160E7
:100B300084BD85B5826085BD85B5816085BD8091A8
:100B40006E00816080936E00109281008091810020
:100B50008260809381008091810081608093810018
:100B6000809180008160809380008091B1008460DA
:100B70008093B1008091B00081608093B00080913B
:100B80007A00846080937A0080917A0082608093FA
:100B90007A0080917A00816080937A0080917A0057
:100BA000806880937A001092C10080913701811192
:100BB00045C010922901109228018FEF80932C01DB
:100BC00080932D0180932E0180932F01809330011B
:100BD0008093310181E080933201109234011092B0
:100BE000330110922B0110922A018091670190919C
:100BF0006801892B31F486E291E09093680180933B
:100C00006701E0912401F0912501309721F086E2FF
:100C100091E09583848386E291E09093250180930F
:100C20002401109236011092350184E191E09093F5
:100C300027018093260181E080933701E09126010E
:100C4000F09127010480F581E02D86E291E009957D
:100C50008FE391E0909329018093280184E090E054
:100C60009093340180933301E0912601F0912701A4
:100C70000284F385E02D86E291E00995009729F141
:100C80009C0140E050E060E472E48FE090E00E945C
:100C90000E07722F632F00915D0110915E0120916C
:100CA0005F0130916001872F962FDA01801791073D
:100CB000A207B30710F4D901C80180935D01909396
:100CC0005E01A0935F01B093600180E090E02FEFA0
:100CD000FC01E15CFE4F10821182228303968C306E
:100CE0009105B1F780915A010E948400DFEF00E086
:100CF00010E0CFEFC0933F011092400110924101EC
:100D000010924201C0934301109244011092450198
:100D100010924601C0934701C093480110924901C7
:100D2000C0934A0180915A010E94840060E375E7F4
:100D300080E090E00E94B50180E090E0FC01E15C81
:100D4000FE4F1082D183D28303968C309105B1F788
:100D500080915A010E94840068EB7BE080E090E083
:100D60000E94B5010115110529F20E940000C2CFB1
:100D7000EAE5F1E08FEF80831282118214861386F8
:100D80008FEF9FEFDC0187839087A187B28708955B
:100D9000DB018F939F930E943407BF91AF91A29F75
:100DA000800D911DA39F900DB29F900D1124089569
:100DB00097FB072E16F4009407D077FD09D00E9408
:100DC0003F0707FC05D03EF4909581959F4F08950D
:100DD000709561957F4F0895A1E21A2EAA1BBB1B47
:100DE000FD010DC0AA1FBB1FEE1FFF1FA217B307F7
:100DF000E407F50720F0A21BB30BE40BF50B661F0D
:100E0000771F881F991F1A9469F7609570958095D0
:100E100090959B01AC01BD01CF010895052E97FB74
:100E20001EF400940E94250757FD07D00E94EC068F
:100E300007FC03D04EF40C9425075095409530954F
:100E400021953F4F4F4F5F4F089590958095709536
:100E500061957F4F8F4F9F4F08950E945907B7FFAD
:100E60000895821B930B08950E945907A59F900D2A
:100E7000B49F900DA49F800D911D11240895AA1B6D
:100E8000BB1B51E107C0AA1FBB1FA617B70710F075
:100E9000A61BB70B881F991F5A95A9F780959095A7
:100EA000BC01CD010895EE0FFF1F0590F491E02DD8
:100EB0000994A29FB001B39FC001A39F700D811D33
:100EC0001124911DB29F700D811D1124911D089553
:0E0ED00081E090E0F8940C946D07F894FFCF49
:100EDE000000000046054605460522051E051B05B9
:100EEE0000000000D8049404920422051E058F040D
:020EFE003C02B4
:00000001FF
